:020000040000FA
:020000000528D1
:08000800080083120730990083
:100010000D309F008316FF23900058309F00FB3067
:100020008500831200308500103050209F149F18E7
:1000300017281E08A200A20EA20C0508A300033078
:10004000A30526202219043A85001D280330220525
:1000500082072D28332839283F28230882070034B7
:100060000034003404342308820700340434043498
:100070000434230882070034043404340034A40117
:10008000050803394B2022195520221D5020A409B0
:100090002408850040288207023405340A341434C9
:1000A000A5005B20A50B51280800A6006430502055
:1000B000A60B56280800C6300000FF3E031D5C2832
:1000C00000000000000008005034653474346534CA
:1000D0002034473472346934663466346934743495
:1000E000683473342034323430343034343420348F
:1000F0002D342034523431343134303435343034CA
:0801000034342E343034323463
:02400E00843FED
:00000001FF
